:10000000000018308A000028FF00030E8301A100C1
:100010000A08A0008A010408A2007708A300780853
:10002000A4007908A5007A08A6007B08A70083131E
:1000300083128C308400001C1F280C183C288C3044
:100040008400801C25288C183F288B1E29280B191A
:100050004228220884002308F7002408F800250815
:10006000F9002608FA002708FB0020088A00210E64
:100070008300FF0E7F0E09008A110A12362B8A11A7
:100080000A12F72B8A110A121F2B0A108A100A1162
:100090008207573457342D343034313420344334CC
:1000A000433453342034433420345334713475345E
:1000B00061347234653420344534783461346D34BD
:1000C00070346C3465342034533474346134723495
:1000D000743469346E34673421340D340A34003496
:1000E0000A108A100A11820752343A3420344534F7
:1000F0006E346334533470346434203425346C34B7
:1001000064343B34203450346F3473342034253419
:100110006C346434203446347734643420342534E9
:1001200064343B34203400340A108A100A118207E8
:100130004C343A34203445346E34633453347034A0
:100140006434203425346C3464343B3420345034EB
:100150006F347334203425346C34643420344634A2
:10016000773464342034253464340D340A34003454
:100170000A108A100A11820720346634203425348C
:100180006C34643420347234653471342034253452
:100190006C34643420346F34753474342034253432
:1001A0006C3464342034643469347234203425343B
:1001B0006C3464340D340A3400340A108A100A1185
:1001C000E43E03188A0A82002034723465347134A4
:1001D000203425346C346434203465346E34633414
:1001E000203425346C34643420346F3475347434E2
:1001F000203425346C3464342034643469347234EB
:10020000203425346C3464340D340A3400340A1438
:100210008A100A11820745346E3463346F346434B3
:1002200065347234203454346534733474340D348A
:100230000A3400340A148A100A11820768346934B7
:100240007434203465346E3474346534723420343C
:1002500074346F342034733474346F3470340D3428
:100260000A3400340A148A100A1182074D346F349C
:1002700074346F34723420345434653473347434C9
:100280000D340A3400340A148A100A1182076834C3
:100290006934743420346B346534793420347434E4
:1002A0006F3420347434753472346E3420346C34CA
:1002B0006534663474342034773468346534653496
:1002C0006C34203466346F34723477346134723471
:1002D00064343A34203400340A148A100A11820734
:1002E00068346934743420346B34653479342034A0
:1002F00074346F3420347434753472346E34203472
:100300007234693467346834743420347734683430
:10031000653465346C34203466346F347234773429
:100320006134723464343A34203400340A148A104C
:100330000A11820768346934743420346B346534AC
:100340007934203474346F34203474347534723416
:100350006E3420346C34653466347434203477342D
:100360006834653465346C34203462346134633409
:100370006B3477346134723464343A34203400346A
:100380000A148A100A1182076834693474342034DC
:100390006B3465347934203474346F3420347434DD
:1003A000753472346E34203472346934673468348E
:1003B0007434203477346834653465346C342034D4
:1003C0006234613463346B3477346134723464344E
:1003D0003A34203400340A148A100A11F23E031809
:1003E0008A0A820068346934743420346B3465348A
:1003F0007934203474346F342034733474346F346B
:1004000070343A34203400340A108A140A118207F6
:100410000D340A3444346F346E3465342E340D3464
:100420000A3400340A108A140A11820753347034D3
:100430006534653464342034723461346D3470341E
:10044000203474346534733474340D340A34003415
:100450000A108A140A1182072D342D343E342034B8
:10046000523465347134753465347334743465349E
:1004700064342034533470346434523420343D3482
:10048000203425346C3464343B3420345334703499
:1004900064344C3420343D34203425346C3464349A
:1004A0000D340A3400340A108A140A1182074434C5
:1004B0006F346E3465342E340D340A3400340A102F
:1004C0008A140A11820750346F34733469347434D7
:1004D00069346F346E342034743465347334743456
:1004E0000D340A3400340A108A140A118207463483
:1004F0007734643420343134203466346F346F34CC
:1005000074340D340A3400340A108A140A11820734
:100510005434753472346E3469346E346734203434
:1005200039343034433443340D340A34003403173F
:100530004E08840083134F1883178018BE2A4E0874
:10054000F8004F08FA004E08D1004F08D200D0083A
:100550000319AC2A0030AD2A0130F8007818B72A08
:10056000510884008313521883170011BD2A5108C3
:1005700084008313521883170015D52A4E08F800FB
:100580004F08FA004E08D1004F08D2005018CF2A69
:10059000510884008313521883170011D52A51087B
:1005A000840083135218831700154E0884008313A8
:1005B0004F188317001DEA2A01304E078400831369
:1005C0004F18831701308007031CE92A840A800A28
:1005D0008403F72A01304E07840083134F188317D2
:1005E000FF3080070318F72A840A800384030A3047
:1005F0004E07840083134F188317800A0F304E076D
:10060000840083134F18831771088000840A7208CE
:100610008000840A73088000840A7408800009300E
:100620004E07840083134F188317001408304E07B9
:10063000840083134F188317800103130034FF30A5
:1006400081000030061A01300317C7000313690840
:100650000317CF00031368080317CE004708D00024
:10066000031397220B118A110A122928FF308F00D9
:100670008E000030861A01300317CD0003136B087B
:100680000317CF0003136A080317CE004D08D000EC
:10069000031397220C108A110A12292894138C1123
:1006A00003175808031393000230941B5E2B8C1D14
:1006B000572B00308316111B01308312F8000034D1
:1006C000831611141118622B403083120317D800BF
:1006D00003134E2303175708D80003134E23831622
:1006E00011151119712B831200342530031753078C
:1006F0008400831354188317840A0008D8008403E5
:100700000008D700D708031D8A2BD808031D8A2BA1
:10071000D501B72B25305307840083135418831752
:10072000840A0008D80084030008D700D81B9F2B38
:10073000D808031DB52B5708733C031CB52B253077
:1007400053078400831354188317840A0008D800C1
:1007500084030008D7008C305707F8005808FA00C7
:100760000318FA0A7808D500B72BFF30D5002730D8
:10077000530784008313541883170018C12B561095
:10078000C22B56145308840083135418831700187F
:10079000CB2B0130D60603136A0803175302031D3F
:1007A000E52B03136B0803175402031DE52B561C9E
:1007B000DD2B0313EC14DF2B03170313EC100317CB
:1007C000550803139B00F12B0317561CEB2B031347
:1007D0006C14ED2B031703136C1003175508031348
:1007E00095006C080317D700031360230034013011
:1007F000F1070318F20A0319F30A0319F40AF50AB8
:100800000319F60A7508C83C031D192CF608031DC8
:10081000192C6F14FC0A0319FD0AF601F5013108C1
:100820000F3C0318B10A831628080F3C0318A80AC6
:100830008312EF1C2E2CEF1069080317D40003134A
:1008400068080317D300031375236B080317D4003C
:1008500003136A080317D300031375238C108A113E
:100860000A122928EB01A030EA008316A014831293
:10087000E9012930E80029141B3083168500FF3078
:100880008600E1308700F0308800FF308900811356
:100890001F149F141F159F1183121F139F17831678
:1008A0009F1383121F14831609122F30F700F71DB0
:1008B000642C073083128101813084008313000887
:1008C000C0390F388000831664008130840000082E
:1008D000C03977048000FF30831281008730900098
:1008E000FF308F008E001830F80004389200FF307F
:1008F00083169200831207110C30970087109D0019
:1009000095019B01EC01A8018B1BA8178B136C08A8
:100910000317D70003136023A81B8B1700008B1647
:1009200083160C148C14C03083128B048316E001E0
:100930006008831245208316E00AF70083120C1A20
:10094000A32C83169E2C9900263083166002031D6B
:10095000982C83128A150A1653280317991BC62C44
:100960009B1FB52C991FC12CB72C991BC52C1B089C
:100970001902031CC52C031DC12C18081A020318E8
:10098000C52C1B0899001A089800E82C1A08003C8E
:10099000F700FA011B08031C1B0FFA027708F80086
:1009A000991FD52CFA1FE12CD72CFA1BE82C19081B
:1009B0007A02031CE82C031DE12C780818020318A6
:1009C000E82C1A0998001B099900980A0319990A3A
:1009D0001808F8001908F900031300340317130866
:1009E0009900120898009B013F309A000313AD2430
:1009F00079080317930078089200283010078400C4
:100A0000831311188317840A0008950084030008D3
:100A100094000030951B013095000030931B01308D
:100A20001506003A03191E2D1D301007840083138C
:100A300011188317840A8001840380012330100772
:100A40008400831311188317840A800184038001B2
:100A5000283010078400831311188317840A1308A1
:100A60008000840312088000031300346908031710
:100A70009100031368080317900093019201031378
:100A8000EE246B080317910003136A080317900004
:100A9000930192010313EE24CF01CE018316C60108
:100AA000C5018312A8018B1BA8178B1369080317B4
:100AB000D400031368080317D30003137523A81B7E
:100AC0008B17A8018B1BA8178B136B080317D40077
:100AD00003136A080317D30003137523A81B8B178E
:100AE000EF140034F701F801F901FA010317A3012B
:100AF000A401A501A6012208210420041F04031952
:100B0000B12D2030A70003109B0D9C0D9D0D9E0D57
:100B1000A30DA40DA50DA60D22082602031D9A2DD6
:100B200021082502031D9A2D20082402031D9A2D59
:100B30001F082302031CAB2D1F08A3022008031C5F
:100B4000200FA4022108031C210FA5022208031C68
:100B5000220FA6020314F70DF80DF90DFA0DA70BDD
:100B6000832D000023308400831703138A150A1293
:100B7000A328B630F700FA01F901F80103171408A9
:100B8000150416041704031DC72DF701D42D0310F7
:100B9000F81BD32D940D950D960D970DFA0DF90DAB
:100BA000F80DF70BC72DF81303138A150A12F9284D
:100BB0000317140803199E2EA000180803199E2E6F
:100BC000A002031CE82D7F30A00703189E2EEE2DF7
:100BD0008130A002031C9E2E03199E2E2008F700D0
:100BE000F801F901FA019F0115089E009E171608E9
:100BF0009D0017089C001930A0001B089C020318D8
:100C0000112E01309D020318112E9E020318112E81
:100C10009F020318112E9F0A9E0A9D0A1B089C071B
:100C2000432E1A089D0203182C2E01309E02031831
:100C30002C2E9F0203182C2E9F0A9E0A1A089D072D
:100C40001B089C07031C432E9D0A031D432E9E0A6E
:100C5000031D432E9F0A432E190880389E02031855
:100C6000422E01309F020318422E9F0A1908803835
:100C70009E071A089D07031C202E9E0A031D202E86
:100C80009F0A202E7A14A00B462E512E03109C0D85
:100C90009D0D9E0D9F0D0310FA0DF90DF80DA10D80
:100CA000FD2D211C592E0310F80CF90CFA0CA10C87
:100CB0005C2EF70303199E2EA11B852E03109C0D9D
:100CC0009D0D9E0D9F0D1B089C020318712E013077
:100CD0009D020318712E9E020318712E9F02031CA1
:100CE000942E1A089D0203187C2E01309E020318D0
:100CF0007C2E9F02031C942E190880389E02031834
:100D0000852E01309F02031C942EFA0A031D942E97
:100D1000F90A031D942EF80A031D942EF70A0319ED
:100D20009E2EF80CF90CFA0C1508A0001908A00664
:100D3000A01F9C2EF817A22EF813A22EF701F8017F
:100D4000F901FA01000003138A150A120E298E30E8
:100D5000F70003171408F7021508F9001608F80041
:100D6000F917F7080319BF2E0310F908031DBB2E4E
:100D7000F8080319BF2EF90CF80CF70BB42E951FC9
:100D8000C62EF809F909F80A0319F90A0000031335
:100D90008A150A121B290317A4010408A3002410B2
:100DA000831B24149D1FDC2EA317231EA30A9C095A
:100DB0009D099C0A03199D0A1D0EF0389F009F078C
:100DC000E23EA000323EA2001D080F39A007A00796
:100DD000A207E93EA100A107A1071C0E0F39A10738
:100DE000A207A10DA20DA209A20D1C080F39A2078E
:100DF0009F0D07309E000A30A207A103031CFC2EA2
:100E0000A107A003031C002FA0079F03031C042FAE
:100E10009F079E03031C082F1E3084008317073092
:100E20002305231384032305031D1D2F231A840A7E
:100E3000231A1D2F2030F7003A2F84072230040296
:100E4000031923170008F700031D2E2F231B2E2F35
:100E5000231A422FA3192E2F2030392FA31F362FEC
:100E60002D30F70084032313A3133A2FA315231265
:100E70003030F707770803130C1A402F03173B2F66
:100E800099000317840A231F1E2F0313003403172E
:100E90001008F801831603136F020318522F6F080E
:100EA000F700662FF70108308312031791008316AD
:100EB0000313EF0DF70D83120317100877020318C1
:100EC000F700F80D910B572F83160313831200348C
:100ED000203083166A1E3030EB006908F700E91FE6
:100EE000782FF709F70A7708E9002D30EB00EA17A9
:100EF0006908EF006430831203179000031347273B
:100F000077088316E90030307807EC006908EF00B5
:100F10000A308312031790000313472730307707F6
:100F20008316EE0030307807ED006B08F700EA1DFD
:100F30009B2FEA1F6A116A1AA82FEA1FC32F6A198A
:100F4000C32F7708EC00EA18C32F7708ED00C32FF2
:100F500030306C02031DC32F7708EC002030EB000B
:100F6000EA1DB62F6A11EA14EA1FEA1030306D024A
:100F7000031DC32F7708ED002030EC00EA1DB62FCB
:100F8000EA10EA1F6A106A1DCD2F6B0883120C1A33
:100F9000CB2F8316C62F99008316EA1CD72F6C0817
:100FA00083120C1AD52F8316D02F990083166A1C32
:100FB000E12F6D0883120C1ADF2F8316DA2F9900A8
:100FC00083166E0883120C1AE72F8316E22F9900FE
:100FD0000034103003179A00F701FA01970C960CB1
:100FE000031CF82F1808F7070318FA0A1908FA075C
:100FF000FA0CF70CF90CF80C9A0BEE2F03130034D3
:101000000930031710078400831311188317001C7D
:101010009529133010079200110893000318930AC2
:101020000F301007840083131118831700089400F1
:10103000840A00089500840A00089600840A0008C3
:1010400097000B30100784008313111883170008D2
:10105000F700840A0008F800840A0008F900840AEE
:101060000008FA0077081402F7007808031C780FCC
:101070003B2815083C281502F8007908031C790F55
:101080004328160844281602F9007A08031C7A0F30
:101090004B2817084C281702FA009B0079089A0081
:1010A00078089900770898001208840083131318B1
:1010B000831718088000840A19088000840A1A0817
:1010C0008000840A1B0880000A3010078400831304
:1010D000111883170008013C0318C22813301007A9
:1010E0009200110893000318930A120884008313D6
:1010F0001318831700089400840A00089500840AD6
:1011000000089600840A000897000A30100784003F
:10111000831311188317000898009A010408990096
:101120001A10831B1A1417089E0016089D00150834
:101130009C0014089B00A201A101A00118089F00B7
:101140008A110313722D8A1503171908840083135B
:101150001A1883177A08980079089700780896007B
:101160007708950012088400831313188317150855
:101170008000840A16088000840A17088000840A08
:101180001808800013301007840083131118831788
:101190008008031DD728840A8008031DD728840AE5
:1011A0008008031DD728840A8008031929291730CD
:1011B00010079200110893000318930A13301007C8
:1011C00084008313111883170008F700840A0008AD
:1011D000F800840A0008F900840A0008FA00970061
:1011E0007908960078089500770894008A1103130F
:1011F000B92D8A15933003179700FC3096004D30B7
:1012000095008A3094007A089B0079089A00780843
:101210009900770898008A110313D82D8A157A0847
:1012200003179700790896007808950077089400CE
:101230008A110313A72E8A1503171208840083133B
:1012400013188317840A79088000840378088000C3
:101250003329173010078400831311188317840A69
:101260008001840380010B30100792001108930065
:101270000318930A0F301007840083131118831783
:101280000008F700840A0008F800840A0008F90042
:10129000840A0008FA0012088400831313188317C5
:1012A00077088000840A78088000840A7908800022
:1012B000840A7A0880000A3010078400831311180A
:1012C00083178001100884008313111883170019F5
:1012D0009429173010079200110893000318930AFD
:1012E000173010078400831311188317840A00082D
:1012F000FA0084030008003CF7007A08031C7A0F08
:10130000832900308429003CFA00770894007A0889
:10131000950012088400831313188317840A150894
:101320008000840314088000BF290830100784005F
:1013300083131118831700080F3C0318BF291330BB
:1013400010078400831311188317E0308000840A8B
:101350000C308000840A8001840A80011730100755
:101360008400831311188317840A80018403800189
:101370000930100784008313111883170014031316
:1013800000340030291901308316E500E6016608B3
:101390008A11831270208A158316E60AF7008312D9
:1013A0000C1AD4298316CF2999000A3083166602B5
:1013B000031DC729103084008312410803179D00C4
:1013C0000313400803179C008A110313CB268A15C8
:1013D0000D308316E70067088A11831270208A1582
:1013E0008316E70AF70083120C1AF8298316F329EB
:1013F0009900133083166702031DEB291030840017
:1014000083122B0803179D0003132A0803179C005F
:101410008A110313CB268A1516308316E800680854
:101420008A11831270208A158316E80AF700831246
:101430000C1A1C2A8316172A99001B30831668027F
:10144000031D0F2A6508E9001F30EA008A11831284
:1014500068278A153B300C1E2B2A990020300C1E61
:101460002F2A99000030831620190130E500E6018B
:1014700066088A11831294208A158316E60AF700FB
:1014800083120C1A452A8316402A99000A308316C3
:101490006602031D382A10308400380883120317AF
:1014A0009D00831603133708831203179C008A11CB
:1014B0000313CB268A150D308316E70067088A11BF
:1014C000831294208A158316E70AF70083120C1AF8
:1014D0006B2A8316662A9900133083166702031D50
:1014E0005E2A103084002208831203179D008316A1
:1014F00003132108831203179C008A110313CB26C0
:101500008A1516308316E80068088A118312942021
:101510008A158316E80AF70083120C1A912A83169B
:101520008C2A99001B3083166802031D842A6508E3
:10153000E9001F30EA008A11831268278A150D30EE
:101540000C1EA02A99000A300C1EA42A990000340F
:1015500003171708190680399B00971FB42A9609AC
:101560009709960A0319970A991FBB2A980999099E
:10157000980A0319990AF801F901F701FA01190803
:10158000031DC52A18080319DF2A10309A0003101A
:10159000960D970DF70DFA0D19087A02031DD22A40
:1015A00018087702031CDB2A1808F702031CFA0349
:1015B0001908FA020314F80DF90D9A0BC72A000056
:1015C0009B1FE72AF809F909F80A0319F90A031316
:1015D0000034253003171007F8001108FA0003182B
:1015E000FA0A780892007A089300193010078400EC
:1015F000831311188317840A0008950084030008D8
:101600009400150897001408960099010930980075
:101610000313A8227808031795007908960012088A
:101620008400831313188317840A16088000840328
:1016300015088000253010078400831311188317C4
:10164000840A00089300840300089200931B302B47
:101650002730100784008313111883170014662B9A
:1016600027301007840083131118831700102530CA
:101670001007F8001108FA000318FA0A7808920017
:101680007A089300253010078400831311188317FC
:10169000840A0008FA0084030008003CF7007A0876
:1016A000031C7A0F552B0030562B003CFA007708AC
:1016B00094007A0895001208840083131318831786
:1016C000840A150880008403140880002530100760
:1016D0008400831311188317840A0008930084037D
:1016E00000089200931B832B1308003C0318832BE4
:1016F000253010078400831311188317840A800192
:101700008403FF3080000313EF1400346F1009309E
:10171000831665078400831366188317001CBF2D8A
:1017200009306507840083136618831700101B3087
:101730006507F8006608FA000318FA0A78088312A9
:10174000031790007A089100283083160313650769
:101750008400831366188317840A00088312031712
:101760009300840300089200173083160313650763
:101770008400831366188317840A0008FA00840320
:1017800000088312031712029400130895007A08C8
:10179000031C7A0F9502150897001408960099010A
:1017A000103098008A110313E9278A157808031767
:1017B0009500790896001008840083131118831788
:1017C000840A160880008403150880001D308316E3
:1017D00003136507F8006608FA000318FA0A780888
:1017E0008312031790007A0891001D3083160313AB
:1017F00065078400831366188317840A0008831220
:10180000031793008403000892001B308316031310
:1018100065078400831366188317840A00088312FF
:10182000031795008403000894001207960013081C
:1018300097000318970A15089707170899001608C4
:10184000980003309B00E8309A008A110313AD24FE
:101850008A15031710088400831311188317840A4C
:10186000790880008403780880001F3083160313F2
:101870006507F8006608FA000318FA0A7808831268
:10188000031790007A08910023308316031365072D
:101890008400831366188317840A000883120317D1
:1018A00093008403000892001B308316031365071E
:1018B0008400831366188317840A0008FA008403DF
:1018C00000088312031712029400130895007A0887
:1018D000031C7A0F950210088400831311188317D4
:1018E000840A1508800084031408800023308316BE
:1018F00003136507F8006608FA000318FA0A780867
:101900008312031790007A0891001B30831603138B
:1019100065078400831366188317840A0008FA0099
:10192000840300088312031792007A0893001008BA
:101930008400831311188317840A1308800084031A
:10194000120880001B30831603136507840083137D
:1019500066188317840A000883120317970084030C
:10196000000896009901083098008A110313E927AE
:101970008A1578088000840A79088000213083164F
:101980006507F8006608FA000318FA0A7808831257
:10199000031790007A089100283083160313650717
:1019A0008400831366188317840A000883120317C0
:1019B0009300840300089200130897001208960011
:1019C00099010C3098008A110313E9278A157908C8
:1019D00003179400780893001408970013089600E2
:1019E0009901103098008A110313E9278A157808A5
:1019F00003179400790895001008840083131118C8
:101A00008317840A150880008403140880001930A5
:101A1000831603136507F8006608FA000318FA0A2C
:101A200078088312031790007A0891001B30831600
:101A3000031365078400831366188317840A00085C
:101A40008312031793008403000892001D3083164D
:101A5000031365078400831366188317840A00083C
:101A6000FA00840300088312031712079400130876
:101A700095000318950A7A0895071F3083160313FB
:101A800065078400831366188317840A0008FA0028
:101A900084030008831203171407960015089700A3
:101AA0000318970A7A0897072130831603136507EE
:101AB0008400831366188317840A0008FA008403DD
:101AC0000008831203171607F8000318FA0A17080C
:101AD000FA07780898007A089900100884008313A0
:101AE00011188317840A19088000840318088000DD
:101AF0001930831603136507F8006608FA00031807
:101B0000FA0A78088312031790007A0891001930B6
:101B10008316031365078400831366188317840AEA
:101B2000000883120317930084030008920013082F
:101B30009700120896009901103098000313A8220C
:101B40007808031793007908940010088400831321
:101B500011188317840A1408800084031308800076
:101B60008316031366088312031791008316031369
:101B700065088312031790000313E922831683126A
:101B800000346A0883166502031DCF2D83126B088B
:101B900083166602031DCF2DFA014C30D02D523032
:101BA000831203179000563003130C1AD92D031714
:101BB000D42D99000317100803130C1AE12D0317F5
:101BC000DC2D99003A300C1EE32D99001930831654
:101BD00065078400831366188317840A000883123C
:101BE000031791008403000890001B308316031331
:101BF00065078400831366188317840A000883121C
:101C0000031793008403000892001D30831603130A
:101C100065078400831366188317840A00088312FB
:101C2000031795008403000894001F3083160313E4
:101C300065078400831366188317840A00088312DB
:101C400003179700840300089600743003130C1ADE
:101C50002B2E0317262E990020300C1E2D2E9900B6
:101C600010308400031711089D0010089C008A1191
:101C70000313CB268A1520300C1E3C2E99007030A1
:101C80000C1E402E990020300C1E442E990010305E
:101C90008400031713089D0012089C008A11031387
:101CA000CB268A1520300C1E532E990069300C1E4D
:101CB000572E990020300C1E5B2E990010308400A6
:101CC000031715089D0014089C008A110313CB26E6
:101CD0008A1520300C1E6A2E990064300C1E6E2E60
:101CE000990020300C1E722E9900103084000317CA
:101CF00017089D0016089C008A110313CB268A152D
:101D00002130831665078400831366188317840ABD
:101D10000008831203179100840300089000283004
:101D20008316031365078400831366188317840AD8
:101D300000088312031793008403000892002530E3
:101D40008316031365078400831366188317840AB8
:101D500000088312031795008403000894002730BD
:101D600083160313650784008313661883170030F6
:101D700000180130831203179701960020300313D7
:101D80000C1AC42E0317BF2E990066300C1EC62EE7
:101D9000990020300C1ECA2E9900103084000317C1
:101DA00011089D0010089C008A110313CB268A1588
:101DB00006300317980018088A110313B8208A15F3
:101DC0000317980AF70003130C1AE82E0317E32EE3
:101DD00099000B3003171802031DDB2E103084000E
:101DE00013089D0012089C008A110313CB268A1544
:101DF0000E300317990019088A110313B8208A15A9
:101E00000317990AF70003130C1A082F0317032F5F
:101E10009900133003171902031DFB2E10308400A4
:101E200015089D0014089C008A110313CB268A15FF
:101E3000163003179A001A088A110313B8208A155E
:101E400003179A0AF70003130C1A282F0317232FDE
:101E500099001B3003171A02031D1B2F103084003A
:101E600017089D0016089C008A110313CB268A15BB
:101E70000D300C1E392F99000A300C1E3D2F990091
:101E8000003420300317A600A201A301A401A5017C
:101E90001D08FA001C08F9001B08F8001A08F700D2
:101EA0000310771C612F1E08A2071F0803181F0FBD
:101EB000A30720080318200FA40721080318210FE7
:101EC000A507A50CA40CA30CA20CFA0CF90CF80C99
:101ED000F70CA60B502F03138A110A16112C0317A7
:101EE0001D0821068039A7009D1F812F9A099B0993
:101EF0009C099D099A0A03199B0A03199C0A031954
:101F00009D0AA11F8E2F9E099F09A009A1099E0A63
:101F100003199F0A0319A00A0319A10AF701F8017E
:101F2000F901FA01A201A301A401A50121082004DD
:101F30001F041E040319CC2F2030A60003109A0D95
:101F40009B0D9C0D9D0DA20DA30DA40DA50D2108AB
:101F50002502031DB52F20082402031DB52F1F08DD
:101F60002302031DB52F1E082202031CC62F1E08C4
:101F7000A2021F08031C1F0FA3022008031C200F2E
:101F8000A4022108031C210FA5020314F70DF80D6C
:101F9000F90DFA0DA60B9E2F0000A71FDA2FF709E7
:101FA000F809F909FA09F70A0319F80A0319F90AED
:101FB0000319FA0A22308400831703138A110A16C0
:021FC000382CBB
:102000003E3083166507840083136618831700101B
:10201000EB08031922282A30650784008313661809
:10202000831767080007840AF8000008FA000318FD
:10203000FA0A6808FA07840378088000840A7A0894
:1020400080002E282A3065078400831366188317C2
:10205000840A680880008403670880006608831289
:10206000031791008316031365088312031790006A
:10207000831603136A08831203179300831603134E
:1020800069088312031792000A120313EE240A163A
:102090002C308316650783120317900083160313F1
:1020A00066088312031791000318910A28308316DB
:1020B000031365078400831366188317840A0008D6
:1020C000FA00840300088312031792007A08930031
:1020D00010088400831311188317840A13088000E2
:1020E00084031208800032308316031365078312BD
:1020F00003179000831603136608831203179100D9
:102100000318910A2830831603136507840083138C
:1021100066188317840A0008831203179300840348
:102120000008920017308316031365078400831399
:1021300066188317840A0008FA00840300088312D3
:10214000031712029400130895007A08031C7A0FF3
:10215000950215089700140896009901063098001A
:102160000A128A150313A8220A168A11780803177F
:1021700095007908960010088400831311188317BE
:10218000840A160880008403150880003230831604
:10219000031365078400831366188317840A0008F5
:1021A000831203179100840300089000911F0F29E8
:1021B00032308316031365078312031790008316CA
:1021C000031366088312031791000318910A323033
:1021D0008316031365078400831366188317840A24
:1021E0000008FA0084030008003CF7007A08031C8A
:1021F0007A0FFC280030FD28003CFA007708831293
:10220000031792007A0893001008840083131118B2
:102210008317840A13088000840312088000323078
:1022200083160313650784008313661883178008D9
:10223000031D5529840A8008031D55293030650780
:102240008400831366188317840A80018403800145
:102250002E30650783120317900083160313660858
:102260008312031791000318910A28308316031371
:1022700065078400831366188317840A0008FA0030
:10228000840300088312031792007A089300100851
:102290008400831311188317840A130880008403B1
:1022A00012088000E1298316031328306507840093
:1022B000831366188317840A00088312031791009A
:1022C0008403000890001730831603136507840009
:1022D000831366188317840A0008FA008403000831
:1022E000F80083120317911F7829FA1F84297A298D
:1022F000FA1B952911087A02031C9529031D8429CC
:1023000078081002031895293030831603136507E7
:102310008400831366188317840AFF3080008403C7
:10232000FA308000A229831203173030831603137A
:1023300065078400831366188317840A8001840369
:10234000063080002E306507831203179000831635
:10235000031366088312031791000318910A1730BC
:102360008316031365078400831366188317840A92
:102370000008831203179300840300089200303092
:102380008316031365078400831366188317840A72
:102390000008FA0084030008831203171207940050
:1023A000130895000318950A7A0895071008840009
:1023B000831311188317840A1508800084031408F6
:1023C0008000383083160313650784008313661872
:1023D0008317840A8001840380013C3065078400F0
:1023E000831366188317840A800184038001831293
:1023F00000348316660883120317910083160313B3
:1024000065088312031790000A128A15031300202F
:102410000A168A110930831665078400831366182B
:102420008317001C562D3630650783120317900062
:102430008316031366088312031791000318910A89
:102440002A308316031365078400831366188317E5
:10245000840A000883120317930084030008920083
:1024600001308316031365078400831366188317EE
:10247000840A0008FA00840300088312031712027A
:102480009400130895007A08031C7A0F950215082A
:102490009900140898009B0180309A000A120313D7
:1024A000AD240A160317100884008313111883172C
:1024B000840A790880008403780880003630831607
:1024C000031365078400831366188317840A0008C2
:1024D0008312031797008403000896009901403087
:1024E00098000A120313E9270A1678088000840A64
:1024F000790880003830831665078312031790002F
:102500008316031366088312031791000318910AB8
:1025100010088400831311188317840A000893009D
:102520008403000892003630831603136507840085
:10253000831366188317840A000883120317950013
:102540008403000894001508970014089600990168
:10255000023098000A120313E9270A1678080317B5
:1025600012079500130896000318960A7908960733
:1025700010088400831311188317840A160880003A
:10258000840315088000383083160313650783120F
:102590000317900083160313660883120317910034
:1025A0000318910A383083160313650784008313D8
:1025B00066188317840A00088312031793008403A4
:1025C00000089200130899001208980003309B003D
:1025D000E8309A000A120313AD240A1603171008F4
:1025E0008400831311188317840A790880008403F8
:1025F000780880003A3083160313650783120317A7
:1026000090008316031366088312031791000318C2
:10261000910A3C3083160313650784008313661800
:102620008317840A000883120317930084030008A9
:1026300092003630831603136507840083136618EF
:102640008317840A0008FA00840300088312031722
:1026500012029400130895007A08031C7A0F950261
:1026600010088400831311188317840A150880004A
:102670008403140880003C3083160313650783121B
:102680000317900083160313660883120317910043
:102690000318910A363083160313650784008313E9
:1026A00066188317840A0008FA008403000883125E
:1026B000031792007A0893001008840083131118FE
:1026C0008317840A130880008403120880003430C2
:1026D00083160313650783120317900083160313F1
:1026E00066088312031791000318910A3630831687
:1026F000031365078400831366188317840A000890
:102700008312031793008403000892003830831665
:10271000031365078400831366188317840A00086F
:10272000FA008403000883120317120794001308A9
:1027300095000318950A7A0895073A308316031313
:1027400065078400831366188317840A0008FA005B
:1027500084030008831203171407960015089700D6
:102760000318970A7A089707100884008313111832
:102770008317840A170880008403160880002E300F
:102780008316031365078400831366188317840A6E
:102790000008FA00840300088312031790007A08E7
:1027A000910092019301911FD72B92039303343030
:1027B0008316031365078400831366188317840A3E
:1027C0000008FA0084030008F7007A08F800F9010D
:1027D000FA01F81FED2BF903FA037A0883120317A5
:1027E0009700790896007808950077089400990179
:1027F000040898001910831B191413089D0012086F
:102800009C0011089B0010089A001708A1001608E8
:10281000A00015089F0014089E000A128A150313D1
:10282000412F0A168A1103171808840083131918F8
:1028300083177A0894007908930078089200770843
:1028400091009601040895001610831B16141408B5
:102850009D0013089C0012089B0011089A00A1011A
:10286000A00120309F009E010A128A1503136F2FCA
:102870000A168A1103171508840083131618831784
:10288000780883160313E8007708E7003E306507F1
:1028900084008313661883170018212D36306507CE
:1028A0008400831366188317840A000883120317B1
:1028B00091008403000890001108FA001008911F8D
:1028C0006A2C1008003CF700FA011108031C110FD4
:1028D000FA02770891007A089200921B732C120872
:1028E000003C031C9C2C831603136808FA0067083D
:1028F000E81F832C6708003CF700FA016808031CF6
:10290000680FFA0277088312031790007A08910083
:10291000911B912C9108031D9C2C1008093C031C51
:102920009C2C3E30831603136507840083136618BE
:1029300083170014831203173230831603136507BD
:1029400084008313661883178008031DAB2C840A48
:1029500080080319F52C323065078400831366184C
:102960008317FF3080070318B82C840A8003840380
:102970002E30650783120317900083160313660831
:102980008312031791000318910A1008840083131F
:1029900011188317840A000893008403000892002A
:1029A000303083160313650784008313661883177A
:1029B000840A0008FA008403000883120317120730
:1029C0009400130895000318950A7A0895071008D3
:1029D0008400831311188317840A15088000840368
:1029E000140880001F2D831603132E3065078312F1
:1029F00003179000831603136608831203179100D0
:102A00000318910A2C30831603136507840083137F
:102A100066188317840A0008FA00840300088312EA
:102A2000031792007A08930010088400831311188A
:102A30008317840A13088000840312088000831619
:102A40000313093065078400831366188317001089
:102A5000193065078400831366188317680883128A
:102A60000317970083160313670883120317960052
:102A70009901253098000A120313E9270A167808ED
:102A80008000840A79088000831666088312031781
:102A900091008316031365088312031790000A122E
:102AA0008A150313E9220A168A1183168312003449
:102AB0006A0883166502031D662D83126B08831650
:102AC0006602031D662DFA014C30672D52308312C9
:102AD0000317900003130C1A6F2D03176A2D99002A
:102AE00050300C1E712D99003A300C1E752D990036
:102AF0003430831665078400831366188317840AAD
:102B000000088312031791008403000890003630F8
:102B10008316031365078400831366188317840ADA
:102B200000088312031793008403000892003830D2
:102B30008316031365078400831366188317840ABA
:102B400000088312031795008403000894003A30AC
:102B50008316031365078400831366188317840A9A
:102B6000000883120317970084030008960074304E
:102B700003130C1ABD2D0317B82D990020300C1E1D
:102B8000BF2D990010308400031711089D00100814
:102B90009C000A120313CB260A1620300C1ECE2DE1
:102BA000990070300C1ED22D990020300C1ED62DAD
:102BB000990010308400031713089D0012089C0030
:102BC0000A120313CB260A1620300C1EE52D99009D
:102BD00069300C1EE92D990020300C1EED2D990056
:102BE00010308400031715089D0014089C000A1279
:102BF0000313CB260A1620300C1EFC2D99006430DE
:102C00000C1E002E990020300C1E042E990010304E
:102C10008400031717089D0016089C000A1203136E
:102C2000CB260A162A30831665078400831366189C
:102C30008317840A00088312031791008403000895
:102C40009000013083160313650784008313661810
:102C50008317840A00088312031793008403000873
:102C600092002530831603136507840083136618CA
:102C70008317840A00088312031795008403000851
:102C800094002730831603136507840083136618A6
:102C90008317003000180130831203179701960044
:102CA000980118080A120313DD200A160317980A60
:102CB000F70003130C1A5E2E0317592E99000530E6
:102CC00003171802031D512E1030840011089D00B7
:102CD00010089C000A120313CB260A1608300317AB
:102CE000990019080A120313DD200A160317990A1E
:102CF000F70003130C1A7E2E0317792E99000D305E
:102D000003171902031D712E1030840013089D0053
:102D100012089C000A120313CB260A161030031760
:102D20009A001A080A120313DD200A1603179A0ADA
:102D3000F70003130C1A9E2E0317992E99001530D5
:102D400003171A02031D912E1030840015089D00F0
:102D500014089C000A120313CB260A161830031716
:102D60009B001B080A120313DD200A1603179B0A97
:102D7000F70003130C1ABE2E0317B92E99001D304D
:102D800003171B02031DB12E1030840017089D008D
:102D900016089C000A120313CB260A160D300C1ECF
:102DA000CF2E99000A300C1ED32E99000034FD015D
:102DB000FC0183166608831203179700831603131A
:102DC00065088312031796009901183098000A12BB
:102DD0000313E9270A1679088316E6007808E50048
:102DE0007D086602031CFA2E031DF92E65087C027D
:082DF000031CF02E83120034D5
:103000001F3083055030F700203084008313800187
:10301000840AF70B0728F101F201F301F401F5012D
:10302000F601F801F901FA01FB01FC01FD01FE01C5
:103030005030F700A030840083138001840AF70B1E
:103040001D286030F7001030840083178001840A47
:10305000F70B262883135930F7009030840083172C
:103060008001840AF70B30288313A00184018313A5
:103070001F30830583161F149F141F159F112030C6
:1030800099002630980090308312980031308316D2
:1030900093002830831294008316941714130A1295
:1030A0008A118312322C0A168A150A128A113625C1
:1030B0000A168A158316E00160080A128A11831223
:1030C00007210A168A158316E00AF70083120C1AE4
:1030D0006B288316662899000E3083166002031D44
:1030E0005C28E00160080A128A1183121A210A166C
:1030F0008A158316E00AF70083120C1A81288316BA
:103100007C289900133083166002031D72288312F5
:1031100032188E288316291CB2288312321C9C2850
:1031200069080317910003136808031790000A1237
:10313000031300200A1632108316291CAD288312AF
:103140006B080317910003136A08031790000A1213
:10315000031300200A16831629100A128312C121B4
:103160000A16831683128C1EBE280A12C1210A1663
:103170008C1EB8281A080D3C0319C128831687280D
:1031800083128316E00160080A128A118312322129
:103190000A168A158316E00AF70083120C1AD22841
:1031A0008316CD2899000C3083166002031DC328B6
:1031B000E00160080A128A11831243210A168A1557
:1031C0008316E00AF70083120C1AE8288316E32816
:1031D0009900243083166002031DD92883128C1AAB
:1031E000F3288316EE288C1EF3281A080D300C1EC7
:1031F000F72899000A300C1EFB289900CF01CE0158
:1032000050148316C601FF30C50047148312EF1413
:103210008316E00160080A128A1183126C210A16D3
:103220008A158316E00AF70083120C1A19298316EF
:1032300014299900253083166002031D0A29831280
:103240008C1A242983161F298C1E24291A080D3054
:103250000C1E282999000A300C1E2C29990083166F
:10326000C601C50147148312CF01FF30CE005014B0
:10327000EF148316E00160080A128A118312962166
:103280000A168A158316E00AF70083120C1A4A29D7
:10329000831645299900253083166002031D3B29BA
:1032A00083128C1A5529831650298C1E55291A0809
:1032B0000D300C1E592999000A300C1E5D29990009
:1032C000CF01CE0150108316C601FF30C500471054
:1032D0008312EF148316E00160080A128A11831228
:1032E000C0210A168A158316E00AF70083120C1A09
:1032F0007B29831676299900263083166002031DE8
:103300006C2983128C1A8629831681298C1E8629A2
:103310001A080D300C1E8A2999000A300C1E8E29BD
:1033200099008316C601C50147108312CF01FF30F3
:10333000CE005010EF148316E00160080A128A11C3
:103340008312EB210A168A158316E00AF70083120E
:103350000C1AAC298316A729990011308316600234
:10336000031D9D2983128C1AB7298316B2298C1E3E
:10337000B7291A088316E00160080A128A1183121D
:1033800004220A168A158316E00AF70083120C1A23
:10339000CB298316C6299900093083166002031DC4
:1033A000BC290A128A11831236250A168A150000D2
:1033B0008316E50165080A128A11831212220A1681
:1033C0008A158316E50AF70083120C1AE929831679
:1033D000E4299900113083166502031DDA29E10101
:1033E0003F30E0006108E3006008E20083126908F2
:1033F0000317910003136808031790008316031343
:103400006108831203179300831603136008831265
:10341000031792000A128A110313EE240A168A1562
:103420006B080317910003136A08031790008316B3
:1034300003136308831203179300831603136208B0
:103440008312031792000A128A110313EE240A163C
:103450008A15FD01FC018316E4016408183C031C75
:10346000562B83126F1C602A6908031791000313FF
:103470006808031790000A12031300200A166B084D
:103480000317910003136A08031790000A1203132D
:1034900000200A1669088316E6008312680883165E
:1034A000E5000A12831286230A166B088316E600CB
:1034B00083126A088316E5000A12831286230A160D
:1034C0007C081F39F700FA0177087A04031D812A66
:1034D0000A12C1210A166B088316E60083126A08D5
:1034E0008316E5000A128312C1250A16690883169D
:1034F000E600831268088316E5000A128312C125CC
:103500000A16FD08031D882A7C08783C0318542BF2
:103510000A12C1210A166B088316E60083126A0894
:103520008316E5000A128312C1250A16690883165C
:10353000E600831268088316E5000A128312C1258B
:103540000A16FD01FC0105308316E0020030031C61
:103550000130E1020530E2020030031C0130E302D9
:10356000E11FC32A6108FF3C031CC32A031DBC2AB8
:103570006008C03C031CC32AE3013F30E20063083B
:10358000E1006208E0008312690803179100031349
:10359000680803179000831603136108831203174A
:1035A00093008316031360088312031792000A1214
:1035B0008A110313EE240A168A156B08031791006B
:1035C00003136A080317900083160313630883121A
:1035D00003179300831603136208831203179200E4
:1035E0000A128A110313EE240A168A158316E501BE
:1035F00065080A128A11831228220A168A15831670
:10360000E50AF70083120C1A072B8316022B990088
:10361000153083166502031DF82A103084006108F6
:10362000831203179D008316031360088312031788
:103630009C000A128A110313CB260A168A15183029
:103640008316E60066080A128A11831228220A16D7
:103650008A158316E60AF70083120C1A312B83169B
:103660002C2B9900213083166602031D222B10306B
:1036700084006308831203179D00831603136208F6
:10368000831203179C000A128A110313CB260A1611
:103690008A150D300C1E4A2B99000A300C1E4E2B39
:1036A00099008316E40A831283162D2AE501650822
:1036B0000A128A11831253220A168A158316E50A02
:1036C000F70083120C1A662B8316612B99000730C2
:1036D00083166502031D572B0A128A1183123625A1
:1036E0000A168A1500008316E50165080A128A1178
:1036F00083125F220A168A158316E50AF7008312E1
:103700000C1A842B83167F2B99000F3083166502C9
:10371000031D752B8312AB01AA018316A201A1011F
:10372000E40164080F3C031CCA2CE50165080A1279
:103730008A11831273220A168A158316E50AF70086
:1037400083120C1AA52B8316A02B99000C3083161C
:103750006502031D962B83120814881469088316CA
:10376000E600831268088316E500E801B230E7003E
:10377000EA013F30E9000130EB008A11831200209A
:103780008A156B088316E60083126A088316E50023
:10379000E801B230E700EA013F30E9000130EB0018
:1037A0008A11831200208A15FD01FC013E306A0750
:1037B000840083136B188317001CE62B3E306807C8
:1037C000840083136918831700181E2C6F1CFE2BAE
:1037D0006B088316E60083126A088316E5008A11D7
:1037E0008312F9218A1569088316E6008312680896
:1037F0008316E5008A118312F9218A15FD08031D3D
:10380000052C7C081E3C03181D2C6B088316E60053
:1038100083126A088316E5008A11831258258A15D7
:1038200069088316E600831268088316E5008A118A
:10383000831258258A15FD01FC01D62B0A128A1124
:1038400036250A168A15000008108316E601023094
:10385000E5008A118312D7268A158316E5016508CB
:103860000A128A11831284220A168A158316E50A1F
:10387000F70083120C1A3E2C8316392C99000E3057
:1038800083166502031D2F2C831208148810690803
:103890008316E600831268088316E500E8012930E4
:1038A000E700EA011F30E9000130EB008A118312C2
:1038B00000208A156B088316E60083126A088316B7
:1038C000E500FF30E800D730E700EA011F30E900EB
:1038D0000130EB008A11831200208A15FD01FC01E2
:1038E0003E306A07840083136B188317001C802CFA
:1038F0003E30680784008313691883170018B82CBA
:103900006F1C982C6B088316E60083126A088316D6
:10391000E5008A118312F9218A1569088316E600E9
:10392000831268088316E5008A118312F9218A152B
:10393000FD08031D9F2C7C081E3C0318B72C6B0848
:103940008316E60083126A088316E5008A11831243
:1039500058258A1569088316E600831268088316BD
:10396000E5008A11831258258A15FD01FC01702C8F
:103970000A128A1136250A168A15000008108316C5
:10398000E6010230E5008A118312D7268A158316D4
:10399000E40A912BE50165080A128A118312532269
:1039A0000A168A158316E50AF70083120C1ADA2C18
:1039B0008316D52C9900073083166502031DCB2C86
:1039C0000A128A11831236250A168A1500000A1275
:0C39D0008A1136250A168A15EC2CED2C05
:02400E00323747
:00000001FF
